:1000000004C1000027C1000025C1000023C1000079
:1000100021C100001FC100001DC100001BC1000064
:1000200019C1000017C100001EC3000087C30000F3
:1000300011C100000FC100000DC100000BC1000084
:1000400009C1000007C1000005C1000003C1000094
:1000500001C10000FFC00000FDC0000042C200005E
:10006000F9C00000F7C00000F5C00000F3C00000B8
:10007000F1C00000EFC00000EDC00000EBC00000C8
:10008000E9C00000E7C00000E5C00000E3C00000D8
:10009000E1C00000DFC00000DDC00000DBC00000E8
:1000A000D9C00000D7C00000D5C000000123022342
:1000B0000423082380230129022904290829402632
:1000C000802640298029102320234023802F402F81
:1000D000202F102F022F012F10292029402C7DFDC9
:1000E0007DFB7DF77DEF7DDF7E7F7EBF7EDF7EEF58
:1000F0007EFD7EFE7DFE0001040506070D0C0B0A49
:1001000009080A0B0C0D0706050401000800010090
:10011000004301120002000055017300220100C8D3
:10012000012100210100B1010900030000E90104DF
:1001300001030904ED011801C13601C02601813611
:100140000180361201000200000040C01685040044
:10015000010001000109027300020100C03209041C
:1001600000000201030000072401000141000624F1
:100170000201010006240202020009240301030116
:10018000020100092403020401010100090504021F
:10019000400000000005250101010905830240001F
:1001A000000000052501010309040100020300000D
:1001B00000092111010001222100070581034000EF
:1001C000010705020320000206C9FF0904A15C75AE
:1001D00008150026FF0095400975810295200976D3
:1001E000910295040976B102C0040309041803546E
:1001F00000650065006E007300790020004D004925
:100200000044004900000000F20611241FBECFEF99
:10021000DAE0DEBFCDBF11E0A0E0B1E0E2E9FEE050
:1002200002C005900D92A431B107D9F711E0A4E105
:10023000B1E001C01D92A737B107E1F712E0CAE0B3
:10024000D2E003C02297FE011ED6C830D107D1F7F5
:10025000DED31DC6D5CE0895089580910101682F83
:1002600070E080910201482F50E08091030190E0FE
:1002700020E030E0FB015FD0FA015DD0FC015BD0F3
:10028000FB015FD0FA015DD0FC015BD02F5F3F4FD7
:100290002830310579F7089590910001891709F404
:1002A000DCCF089585E291E060E0B5C38CE291E097
:1002B00090936701809366018BE291E090936901CE
:1002C000809368018CE491E09093750180937401B0
:1002D000809101011FD0809102011CD08091030107
:1002E00019D080910101E82FF0E025D08091020122
:1002F000E82FF0E020D068E873E180E090E031D1B1
:1003000080910101E82FF0E01CD080910201E82FDC
:10031000F0E017C0893170F4ECEAF0E0880FE80FE4
:10032000F11D9591E491F0E02FB7F8948181892B2C
:1003300081832FBF0895E93150F4EE0FE855FE4F49
:100340000994E93120F4EE0FE652FE4F0994089526
:10035000289A0895299A08952A9A08952B9A08951B
:100360002F9A6AC0589A58C0599A08955A9A08956F
:100370005B9A0895469A66C0479A6AC05E9A089545
:100380005F9A6CC02C9A08952D9A4AC02E9A4EC03E
:100390008F9A08958E9A08958D9A08958C9A08954B
:1003A000899A0895889A08955C9A08955D9A0895A7
:1003B000769A089528980895299808952A98089576
:1003C0002B9808952F9838C0589826C059980895AA
:1003D0005A9808955B980895469834C0479838C055
:1003E0005E9808955F983AC02C9808952D9818C08B
:1003F0002E981CC08F9808958E9808958D98089512
:100400008C98089589980895889808955C9808951F
:100410005D98089576980895E4B5EF7DE4BD08955C
:10042000E0918000EF77E09380000895E0918000F4
:10043000EF7DE09380000895E0918000E77FE093F6
:1004400080000895E0919000EF77E0939000089588
:10045000E091C000EF77E093C0000895E091C20002
:10046000E77FE093C20008951DBA109268001CBC9B
:1004700010BE1FBA10927A0010926E0010926F0098
:1004800010927100109272001092C900ECEBF0E033
:10049000108214B817B81AB81DB810BA108215B85F
:1004A00018B81BB81EB811BA0895F89480E29EE4FB
:1004B0000197F1F781E08093E00080E28093D8001B
:1004C00080E69AEE0197F1F7CFDF0C94003FFFCF63
:1004D000F894CADF80E69AEE0197F1F70C940000D9
:1004E000FFCF8F938FB78F9380911C018D5F8D37D6
:1004F000D0F480931C01809118018F5F80931801C4
:10050000D8F0809119018F4F80931901A8F0809144
:100510001A018F4F80931A0178F080911B018F4F41
:1005200080931B0109C08D5780931C018091180195
:100530008E5F8093180128F7809114018C5F80935F
:10054000140158F0809115018F4F8093150128F008
:10055000809116018F4F809316018F918FBF8F91DD
:1005600018959B01AC0114D0FB010CC011D06E1B7F
:100570007F0B685E7340D0F32150304040405040C4
:10058000E851FC4F211531054105510579F70895D2
:100590000FB6F89466B515B27091140180911501EB
:1005A000909116010FBE10FE05C06F3F19F07C5FE1
:1005B0008F4F9F4F11240024660F001C660F001CF4
:1005C00070290895F894E1E6F0E020E82083108295
:1005D00083E084BD85BDEEE6F0E0808181608083AC
:1005E00091E09093800082E080938100909390004E
:1005F000809391008093C00084E08093C100909329
:10060000C2009093C3001092C40086E880937A00E1
:1006100020937B0010927E0010927D0002D078948F
:1006200008958091D80087FF02C085FF1BC081E03C
:100630008093D70080EA8093D80082E189BD09B415
:1006400000FEFDCF80E98093D8001092E000109268
:10065000770110927801109279011092E1008CE0FC
:100660008093E20008951F920F920FB60F9211240B
:100670008F939F938091E1001092E100982F83FF68
:100680000FC01092E90081E08093EB001092EC0023
:1006900082E38093ED0088E08093F0001092770170
:1006A00092FF24C080917701882301F18091790124
:1006B000882391F0815080937901882369F481E047
:1006C0008093E90002C01092F1008091E80085FD5E
:1006D000FACF8AE38093E80083E08093E900809179
:1006E000F200882319F08AE38093E80090FF0CC0A1
:1006F00080E18093E2001092770181E0809378019D
:1007000080EA8093D80019BC80917801882379F021
:1007100094FF0DC082E189BD09B400FEFDCF80E9E0
:100720008093D8008DE08093E200109278019F9131
:100730008F910F900FBE0F901F9018951F920F92E0
:100740000FB60F9211242F933F934F935F936F93A4
:100750007F938F939F93AF93BF93EF93FF931092E9
:10076000E9008091E80083FF3EC13091F100909153
:10077000F1004091F1005091F1006091F100709111
:10078000F100A091F100B091F10082EF8093E800B8
:10079000963009F044C0EDE0F1E020E085919591BC
:1007A0008417950711F0359617C085919591861796
:1007B000970711F0339610C0259135914491CD01E2
:1007C000AF3FB10519F010F08FEF90E0841708F4F7
:1007D000482FF9015EEF04C02F5F2630F9F603C100
:1007E0008091E800282F30E0C90185709070892B36
:1007F000B9F322FDFBC0242F413408F020E4922FEE
:1008000004C085918093F10091509923D1F7421B48
:100810005093E800442321F7203411F3E7C09530CA
:1008200061F48EEF8093E8008091E80080FFFCCFB8
:10083000842F80688093E300D9C09930F9F4332382
:1008400009F06FC040937701109279018EEF809389
:10085000E800E7E3F1E091E09093E900859180936F
:10086000EB00882331F085918093EC008591809393
:10087000ED009F5F953081F78EE14EC0983061F4B6
:10088000303809F04EC08091E80080FFFCCF8091A5
:1008900077018093F1001BC09923E9F48091E8006F
:1008A00080FFFCCF323811F080E00DC06093E9008A
:1008B0008091EB0090E025E0969587952A95E1F7E9
:1008C00081701092E9008093F1001092F1008EEF98
:1008D0008093E8008BC0913011F0933011F53230E5
:1008E00001F541155105E9F4262F2F77822F81500C
:1008F0008630B8F48EEF8093E8002093E9009330BF
:1009000009F471C089E18093EB0081E090E002C0BE
:10091000880F991F2A95E2F78093EA001092EA0067
:1009200065C06130710509F052C0913019F5313A56
:1009300009F059C04A2F5EEF8091E800282F30E07F
:10094000C90185709070892BB9F322FD4FC0942F97
:10095000413408F090E4892F03C01092F1008150D7
:100960008823D9F7491B5093E800442329F7903492
:1009700019F33CC0993059F53132A9F54050534034
:1009800091F5149781F58091E80082FFFCCF90915A
:10099000F1002091F1003091F1004091F1008BEFD6
:1009A0008093E8008EEF8093E800993A39F425347B
:1009B000D1F4323CC1F44B36B1F477DD9B3899F475
:1009C000253C89F43D3179F4403769F40BC0993CFA
:1009D00051F4303441F48EEF8093E8008091E800C8
:1009E00080FFFCCF75DD81E28093EB00FF91EF91FA
:1009F000BF91AF919F918F917F916F915F914F9137
:100A00003F912F910F900FBE0F901F901895DADD38
:100A10004DDC48DCFECFFF920F931F93CF93DF9303
:100A2000EC019FB7F89480917701882311F49FBF60
:100A300030C184E08093E9002BE68091E80085FDD9
:100A400007C082FF03C02093E800F7CF9FBF20C1FB
:100A50002091F1003091F1000091F100F090F1004F
:100A60008091E80085FD03C08BE68093E8009FBF7E
:100A7000922F9F70892F8850883008F0AFC0132FB5
:100A80001F70662319F0611709F002C1832F807F60
:100A9000983059F4803809F0FBC01982CF5BDF4FE2
:100AA000E881F981C154D0402BC09930E1F48039FC
:100AB00009F0EEC0FF2049F081E08983CD5BDF4F74
:100AC000E881F981C354D0401BC01982CF5BDF4F4E
:100AD000E881F981C154D040309709F47BC0812F5F
:100AE000602F40E013C09A3099F4803A09F0D0C0EA
:100AF00082E08983CB5BDF4FE881F981C554D04028
:100B0000309709F467C0812F602F4F2D099562C07F
:100B10009B3061F4803B09F0BBC083E08983C95BF3
:100B2000DF4FE881F981C754D040EACF9C3061F4AF
:100B3000803C09F0ADC084E08983C75BDF4FE8816A
:100B4000F981C954D0400DC09D3089F4803D09F031
:100B50009FC085E08983C55BDF4FE881F981CB5475
:100B6000D0403097B9F1812F602F099533C09E3066
:100B7000F9F4803E09F08CC086E08983C35BDF4FC7
:100B8000E881F981CD54D040309721F16F2D70E08C
:100B90006F7770707695762F662777956795802F9B
:100BA00090E08F779070682B792B812F099512C078
:100BB0009F3009F06DC0803F09F06AC088E08983EA
:100BC000C15BDF4FE881F981CF54D040309711F0FD
:100BD000832F099518830A83FB8258C0943021F52E
:100BE000DE01A05CBF4F8C918C3330F4FE01E80F26
:100BF000F11D34838F5F8C93DE01A05CBF4F8C911D
:100C00008C3330F4FE01E80FF11D04838F5F8C9369
:100C1000FE01E05CFF4F80818C33D0F5C80FD11D01
:100C2000FC828F5F808334C0892F8550833080F5AC
:100C3000DE01A05CBF4F8C918C3330F4FE01E80FD5
:100C4000F11D34838F5F8C93963060F0DE01A05CE1
:100C5000BF4F8C918C3330F4FE01E80FF11D0483FB
:100C60008F5F8C93973061F4DE01A05CBF4F8C9155
:100C70008C3330F4FE01E80FF11DF4828F5F8C930A
:100C8000FE01E05CFF4F80818A83108281E001C019
:100C900080E0DF91CF911F910F91FF9008952FB7C2
:100CA000F89480917701882341F082E08093E900F5
:100CB0003BE68091E80085FD03C02FBF90E00FC0A8
:100CC0009091F100992319F43093E800F2CF8091CC
:100CD000E80085FD03C08BE68093E8002FBF892FD5
:100CE000089520917601222349F4D9DF882319F44D
:100CF0002FEF3FEF04C080937601282F30E0C90129
:100D0000089520917601222319F01092760107C0F0
:100D1000C6DF882319F42FEF3FEF02C0282F30E001
:100D2000C90108959C0180917601882349F4C90185
:100D3000B6DF882319F420E030E004C08093760108
:100D400021E030E0C901089580917701882371F096
:100D50009FB7F89482E08093E9002BE602C02093CD
:100D6000E8008091E80085FDFACF9FBF10927601E0
:100D70000895FC0180917701882371F12FB7F894D1
:100D800081E08093E9009091E400975E31E08091EA
:100D9000E80085FD0EC02FBF8091E4008917E1F0C7
:100DA000809177018823C1F02FB7F8943093E90040
:100DB000EECF6093F1008091E80085FD06C08AE3E4
:100DC0008093E8001092790103C084E08093790158
:100DD0002FBF21E030E004C081E0828320E030E0DA
:100DE000C9010895EDE1F1E088E0DF011D928A95E7
:100DF000E9F710921F0188EE93E0A0E0B0E0809345
:100E0000200190932101A0932201B093230110921D
:100E1000240188E091E090931E0180931D01E5E29A
:100E2000F1E081E5DF011D928A95E9F70895CF92FF
:100E3000DF92EF92FF920F931F93CF93DF937C018A
:100E40006B018A01C0E0D0E00FC0D6016D916D0149
:100E5000D701ED91FC910190F081E02DC70109953A
:100E6000C80FD91F015010400115110571F7CE01AF
:100E7000DF91CF911F910F91FF90EF90DF90CF9076
:100E80000895EE0FFF1F0590F491E02D0994F8945A
:020E9000FFCF92
:100E9200F80B0C0100000000B90617079206810644
:040EA2007106A4062B
:00000001FF
